:020000040800F2
:1000000010300020CD010008B12B00082B2400087F
:10001000812B000881040008ED3700080000000073
:10002000000000000000000000000000E52F0008B4
:100030007D05000800000000B52B0008B93000085D
:10004000E7010008E7010008E7010008E7010008F0
:10005000E7010008E7010008E7010008E7010008E0
:10006000E7010008E7010008E7010008E7010008D0
:10007000E7010008E7010008E7010008E7010008C0
:1000800041050008E7010008E7010008E701000852
:10009000E7010008E7010008E7010008E7010008A0
:1000A000E7010008E7010008E7010008E701000890
:1000B000C5300008E7010008E7010008E701000873
:1000C000E7010008E7010008E7010008E701000870
:1000D000E7010008CD370008DD370008E701000818
:1000E000E7010008E7010008E7010008E701000850
:1000F000E7010008E7010008E7010008E701000840
:10010000E7010008E7010008E7010008E70100082F
:10011000E7010008E7010008E7010008E70100081F
:10012000E7010008E7010008E7010008E70100080F
:1001300000F002F800F03AF80AA090E8000C8244BF
:100140008344AAF10107DA4501D100F02FF8AFF29C
:10015000090EBAE80F0013F0010F18BFFB1A43F0A5
:10016000010318470053000020530000103A24BF39
:1001700078C878C1FAD8520724BF30C830C144BF0C
:1001800004680C607047000000230024002500264E
:10019000103A28BF78C1FBD8520728BF30C148BFEA
:1001A0000B6070471FB51FBD10B510BD00F0E8F81B
:1001B0001146FFF7F7FF03F0E5FD00F006F903B481
:1001C000FFF7F2FF03BC03F0BBFB000009488047C8
:1001D00009480047FEE7FEE7FEE7FEE7FEE7FEE729
:1001E000FEE7FEE7FEE7FEE704480549054A064B41
:1001F00070470000C130000831010008102A0020BB
:1002000010300020102C0020102C00207047B2F17C
:1002100020030AD5C2F1200320FA02F001FA03F309
:1002200021FA02F140EA0300704721FA03F04FF08F
:1002300000017047032A40F2308010F0030C00F0F8
:10024000158011F8013BBCF1020F624498BF11F810
:1002500001CB00F8013B38BF11F8013BA2F10402C9
:1002600098BF00F801CB38BF00F8013B11F0030341
:1002700000F02580083AC0F0088051F8043B083AA5
:1002800051F804CBA0E80810F5E7121D5CBF51F847
:10029000043B40F8043BAFF30080D20724BF11F8C1
:1002A000013B11F801CB48BF11F8012B24BF00F826
:1002B000013B00F801CB48BF00F8012B704710B597
:1002C000203AC0F00B80B1E81850203AA0E818504E
:1002D000B1E81850A0E81850BFF4F5AF5FEA027C0F
:1002E00024BFB1E81850A0E8185044BF18C918C07E
:1002F000BDE810405FEA827C24BF51F8043B40F81F
:10030000043B08BF7047D20728BF31F8023B48BF03
:1003100011F8012B28BF20F8023B48BF00F8012B41
:1003200070474FF0000200B51346944696462039B8
:1003300022BFA0E80C50A0E80C50B1F12001BFF49E
:10034000F7AF090728BFA0E80C5048BF0CC05DF804
:1003500004EB890028BF40F8042B08BF704748BF52
:1003600020F8022B11F0804F18BF00F8012B7047C6
:10037000704770477047704700487047B0290020A9
:100380007546FFF7F9FFAE4605006946534620F073
:100390000700854618B020B5FFF726FFBDE82040CE
:1003A0004FF000064FF000074FF000084FF0000B31
:1003B00021F00701AC46ACE8C009ACE8C009ACE8E4
:1003C000C009ACE8C0098D46704710B50446AFF3CC
:1003D00000802046BDE81040FFF7F1BE00200A492A
:1003E00000BF03E00A5C094B1A54401CB0F5486F8B
:1003F000F8D3D1F8802C054BC3F8802CD1F8842C8D
:10040000C3F8842C7047000000F00308A8100020F7
:1004100010B540F244620249024800F0CBF910BD29
:10042000A810002000F0030810B50B480068401C1D
:10043000094908600846006844F62061884209D3EB
:1004400008460549086000BF00220121034801F069
:1004500009F800BF10BD00002C000020000C014076
:1004600010B500BF01221146034800F0FBFF00BF9A
:1004700000200249086010BD000C01402C00002043
:1004800000BFFEE7F0B502460C46FF21FF2509E05C
:1004900012F8016B86EA0103084EF65C86EA050154
:1004A000074EF55C261EA4F10107BCB2F0D1084648
:1004B0004FF6FF7606EA00202843F0BD645200089C
:1004C00064530008F0B505460C46A01E2E5C4FF69E
:1004D000FF7000EA0626601E285C0643A01E81B25B
:1004E0002846FFF7CFFF0746BE4201D10120F0BDED
:1004F0000020FCE770B500BFD52003F09BF900BFDA
:100500000021084602F0BCFD002416E000250DE0A5
:10051000002003F0C5F9002003F0C2F9002003F029
:10052000BFF9002003F0BCF9681C85B2142DEFDB85
:10053000002003F0B5F9601C84B2A02CE6DB70BD8E
:1005400010B5024800F0AAFA10BD000020100020EB
:1005500030B590F840500124AC40C56B6C60046825
:1005600063604468102C04D10468A2600468E160F0
:1005700003E00468A1600468E26030BD70470000D9
:100580002DE9F84F81460F46904630A00068009054
:1005900000BFD52003F04EF900BFB9F1A00F01D87C
:1005A000A02F01D9BDE8F88FC9F1A00040080321B0
:1005B000B0FBF1F000F0FF0AC7F1A00007EB50001C
:1005C00000F0FF0B4FEAD90600243BE0ABEB040040
:1005D000C1B2504602F054FD00252CE004FB065148
:1005E00018F80110C943C1F381111DF8010003F08F
:1005F00057F904FB065118F80110C943C1F3011162
:100600001DF8010003F04CF904FB065118F8011025
:10061000C943C1F381011DF8010003F041F904FB56
:10062000065118F80120032191431DF8010003F041
:1006300037F9681CC5B2B542D0D3002003F030F9B9
:10064000601CC4B2BC42C1D300BFABE7000FF0FFD7
:100650000021074AD1610749096941F00401054AAF
:1006600011611146096941F04001116170470000B4
:1006700068010020002002400021074AD16107499B
:10068000096941F00201054A116111464861096991
:1006900041F04001116170476801002000200240D4
:1006A0000022054BDA61054A126942F00102034B50
:1006B0001A6101807047000068010020002002409C
:1006C00000201E49C96801F0100139B11C49C969EF
:1006D00041F002011A4AD16140F010001749C9687F
:1006E00001F0040139B11649C96941F00101144A08
:1006F000D16140F004001149C96901F0010169B1FB
:100700000F49C96941F004010D4AD16100BF0B498D
:10071000C96921F00101094AD16100BF00BF40F25F
:100720000111884206D10549C96921F00101034A36
:10073000D16101E00149C86000BF7047002002405C
:100740006801002070B5044600F092FE054609E0FD
:10075000601C38B124B100F08BFE401BA04201D9CF
:10076000032070BD1248C06800F001000028EFD1DE
:100770000F48C06800F0200020B100BF20200C49C5
:10078000C86000BF0A48C06800F0100048B90848B7
:10079000C06900F0010020B90548C06800F00400FD
:1007A00018B1FFF78DFF0120DBE70020D9E700003B
:1007B000002002402DE9F74F88B005469046A5F18C
:1007C0000060079007984FEAD02A4FF0006000EBD6
:1007D000CA26A81B06904FEA480705950698384494
:1007E0004FEAD02B4FF000090020009006983844C3
:1007F000C0F30A0008B10BF1010BB5F1006F03D390
:10080000E8192549884203D301200BB0BDE8F08FD9
:10081000B6F1006F02D32048864201D30120F4E7ED
:1008200000F056FC0598C11906F5006081422ED3F0
:10083000002414E0002001900396012004906946F2
:1008400001A800F08BFB8146B9F1000F03D000F046
:10085000DDFB4846D9E706F50066601C84B25C45BE
:10086000E8D3002410E0099830F814C005EB4401E7
:1008700062460023012000F0D3FB8146B9F1000F4E
:1008800000D003E0601C84B24445ECDB00BF00F004
:10089000BDFB4846B9E700000000040801460022FD
:1008A00091F82100022808D00420886300BF0020AE
:1008B00081F8200000BF012070470868006820F020
:1008C0000E000B6818600868006820F001000B68D3
:1008D000186091F8403001209840CB6B586001209F
:1008E00081F8210000BF002081F8200000BF1046E1
:1008F000E2E7000070B50446002594F821000228C4
:1009000003D00420A0630125C1E02068006820F026
:100910000E00216808602068006820F0010021684E
:1009200008605C492068884252D95A497839206861
:10093000884201D1012047E0564964392068884245
:1009400001D1102040E0534950392068884201D13C
:10095000801539E04F493C392068884201D1801424
:1009600032E04C4928392068884202D14FF4803067
:100970002AE0484914392068884202D14FF4801097
:1009800022E044492068884201D140041CE04249E9
:100990002068884201D1012016E03F4914312068C7
:1009A000884201D110200FE03B492831206888425D
:1009B00001D1801508E038493C312068884201D1D6
:1009C000801401E04FF480303349091F086051E082
:1009D000304978392068884201D1012047E02D490B
:1009E00064392068884201D1102040E029495039FB
:1009F0002068884201D1801539E026493C392068B9
:100A0000884201D1801432E0224928392068884286
:100A100002D14FF480302AE01E4914392068884200
:100A200002D14FF4801022E01A492068884201D197
:100A300040041CE018492068884201D1012016E0DA
:100A4000154914312068884201D110200FE0124965
:100A500028312068884201D1801508E00E493C31D8
:100A60002068884201D1801401E04FF480300949A8
:100A700080394860012084F8210000BF002084F8FC
:100A8000200000BF606B10B12046616B884728468C
:100A900070BD0000800002400804024070B50446AA
:100AA000E06B05682068066894F8401004208840D0
:100AB0002840002875D006F004000028FAD02068ED
:100AC000006800F0200028B92068006820F00400C9
:100AD00021680860D5492068884254D9D3497839BB
:100AE0002068884201D1042049E0D0496439206857
:100AF000884201D1402042E0CC49503920688842E8
:100B000001D100153BE0C9493C392068884202D137
:100B10004FF4804033E0C54928392068884202D12B
:100B20004FF480202BE0C14914392068884202D15B
:100B30004FF4800023E0BD492068884201D1C00401
:100B40001DE0BB492068884201D1042017E0B84964
:100B500014312068884201D1402010E0B449283186
:100B60002068884201D1001509E0B1493C31206874
:100B7000884202D14FF4804001E04FF48020AC491C
:100B8000091F086054E0A94978392068884201D1DA
:100B900004204AE0A54964392068884202D14020F7
:100BA00043E04CE0A14950392068884201D100154A
:100BB0003BE09E493C392068884202D14FF4804096
:100BC00033E09A4928392068884202D14FF48020C6
:100BD0002BE0964914392068884202D14FF48000F6
:100BE00023E092492068884201D1C0041DE0904969
:100BF0002068884201D1042017E08D491431206813
:100C0000884201D1402010E089492831206888427B
:100C100001D1001509E086493C312068884202D1A3
:100C20004FF4804001E04FF48020804980394860D3
:100C3000E06A002802D02046E16A8847F4E094F890
:100C40004010022088402840002871D006F00200A1
:100C50000028FAD02068006800F0200040B9206821
:100C6000006820F00A0021680860012084F8210053
:100C70006E492068884254D96C4978392068884286
:100C800001D1022049E0694964392068884201D1D4
:100C9000202042E0654950392068884201D1401542
:100CA0003BE062493C392068884202D14FF4005051
:100CB00033E05E4928392068884202D14FF4003081
:100CC0002BE05A4914392068884202D14FF40010B1
:100CD00023E056492068884201D180041DE0544930
:100CE0002068884201D1022017E051491431206860
:100CF000884201D1202010E04D49283120688842E7
:100D000001D1401509E04A493C312068884202D1AE
:100D10004FF4005001E04FF400304549091F0860CE
:100D200054E0424978392068884202D102204AE0E2
:100D300057E03E4964392068884201D1202042E0D2
:100D40003A4950392068884201D140153BE0374983
:100D50003C392068884202D14FF4005033E03349D7
:100D600028392068884202D14FF400302BE02F4907
:100D700014392068884202D14FF4001023E02B4937
:100D80002068884201D180041DE0294920688842FA
:100D900001D1022017E0264914312068884201D190
:100DA000202010E0224928312068884201D14015D6
:100DB00009E01F493C312068884202D14FF40050BD
:100DC00001E04FF4003019498039486000BF00202D
:100DD00084F8200000BFA06A30B32046A16A88478B
:100DE00022E094F84010082088402840E0B106F046
:100DF0000800C8B12068006820F00E002168086073
:100E000094F8401001208840E16B48600120A06305
:100E100084F8210000BF002084F8200000BF206B70
:100E200010B12046216B884770BD00008000024051
:100E3000080402400146002209B9012070471E4BF8
:100E4000086898420BD21D4B0868C01A1423B0FBE7
:100E5000F3F08000086419480838C8630AE0164BAC
:100E60000868C01A1423B0FBF3F08000086412482D
:100E70000838C863022081F821000868026843F638
:100E8000F0708243D1E901031843CB6818430B6922
:100E900018434B6918438B691843CB6918430243C5
:100EA0000868026000208863012081F8210000208A
:100EB00081F8200000BFC1E708040240080002409A
:100EC0002DE9F04104460D4616461F464FF0000836
:100ED00000BF94F82000012802D10220BDE8F08173
:100EE000012084F8200000BF94F8210001282CD1B3
:100EF000022084F821000020A0632068006820F010
:100F00000100216808603B46324629462046FFF72B
:100F10001FFBE06A30B12068006840F00E002168D5
:100F200008600BE02068006820F004002168086079
:100F30002068006840F00A002168086020680068A6
:100F400040F001002168086006E000BF002084F83E
:100F5000200000BF4FF002084046BFE72DE9F041F6
:100F600004460E460127002500BF2648007E0128C2
:100F700002D10220BDE8F08101202249087600BF9D
:100F80002068022813D14CF25030FFF7DBFB90BBF6
:100F90000120FFF75DFB4CF25030FFF7D3FB074613
:100FA0001948006920F004001749086123E04CF259
:100FB0005030FFF7C7FBF0B94FF0FF303060A56845
:100FC00012E02846FFF758FB4CF25030FFF7BAFB0F
:100FD00007460D48006920F002000B4908610FB177
:100FE000356007E005F50065D4E9021001EBC0208B
:100FF000A842E6D800BF00BF00200249087600BF23
:101000003846B7E768010020002002400348006925
:1010100040F0800001490861002070470020024034
:101020002DE9FE4F05468B461746984601260024BB
:101030000020029000BF2448007E012802D1022037
:10104000BDE8FE8F01202049087600BF4CF25030E9
:10105000FFF778FB064686BB012D02D101200290E6
:1010600006E0022D02D10220029001E0042002904D
:1010700000241EE02201B946C24648465146FFF709
:10108000C6F880B20190022000FB04B000900199E4
:10109000FFF706FB4CF25030FFF754FB06460B48B7
:1010A000006920F001000949086106B104E0601CF4
:1010B000C4B202988442DDDB00BF00BF00200249B9
:1010C000087600BF3046BBE76801002000200240E0
:1010D00000200849096901F0800151B10649054A1B
:1010E0005160064951601146096901F0800101B162
:1010F000012070470020024023016745AB89EFCDF6
:101100002DE9F847024600239C467BE14FF0010899
:1011100008FA03F4D1F8008008EA0400A0427DD167
:10112000DFF8F4A2D1F80480A8EB0A09D0453AD040
:1011300014DCB8F1030F50D009DCB8F1000F31D046
:10114000B8F1010F1CD0B8F1020F49D120E0B8F17D
:10115000110F18D0B8F1120F42D11EE0B9F5881F57
:1011600025D006DCB9F5803F20D0B9F5801F37D1F6
:101170001AE0B9F5001F18D0B9F5041F30D117E0F7
:10118000D1F80CC02DE0D1F80C8008F1040C28E057
:10119000D1F80C8008F1080C23E0D1F80C8008F19C
:1011A0000C0C1EE000BF00BF00BF00BF00BF00BFAF
:1011B000D1F80880B8F1000F02D14FF0040C0BE019
:1011C000D1F80880B8F1010F03D14FF0080C146179
:1011D00002E04FF0080C546103E04FF0000C00E017
:1011E00000BF00BFFF2801D8904601E002F10408CB
:1011F0004646FF2802D84FEA830803E0A3F1080817
:101200004FEA88084746D6F800804FF00F0909FAE0
:1012100007F928EA09080CFA07F900E07AE048EA39
:101220000908C6F80080D1F8048008F08058B8F1A9
:10123000805F6FD100BFDFF8E481D8F8188048F0F4
:101240000108DFF8D891C9F81880C846D8F8188086
:1012500008F00108CDF8008000BF00BF4FEAB938A0
:101260004FEA930958F829504FEA83784FEA1879E2
:101270004FF00F0808FA09F825EA0805DFF8A08101
:10128000424502D14FF0000824E0DFF89881424542
:1012900002D14FF001081DE0DFF88C81424502D1F8
:1012A0004FF0020816E0DFF88481424502D14FF08A
:1012B00003080FE0DFF87881424502D14FF00408BF
:1012C00008E0DFF87081424502D14FF0050801E0E7
:1012D0004FF006084FEA83794FEA197908FA09F8BE
:1012E00048EA0505DFF850814FEA930948F829508C
:1012F000D1F8048008F48018B8F5801F0BD1DFF80E
:101300003C81D8F8008048EA0008DFF83091C9F83D
:1013100000800AE075E0DFF82481D8F8008028EA30
:101320000008DFF81891C9F80080D1F8048008F4AB
:101330000018B8F5001F0ED1DFF8008108F104088D
:10134000D8F8008048EA0008DFF8F09009F10409B5
:10135000C9F800800DE0DFF8E48008F10408D8F84F
:10136000008028EA0008DFF8D49009F10409C9F8E0
:101370000080D1F8048008F40038B8F5003F0ED1A1
:10138000DFF8B880A8F10408D8F8008048EA00081F
:10139000DFF8A890A9F10409C9F800800DE0DFF892
:1013A0009C80A8F10408D8F8008028EA0008DFF83B
:1013B0008C90A9F10409C9F80080D1F8048008F4E0
:1013C0008038B8F5803F0ED1DFF87080A8F10808AA
:1013D000D8F8008048EA0008DFF86090A9F1080911
:1013E000C9F800800DE0DFF85480A8F10808D8F8AB
:1013F000008028EA0008DFF84490A9F10809C9F83C
:1014000000805B1CD1F8008028FA03F8B8F1000FC7
:101410007FF47CAEBDE8F887000011100010024098
:1014200000080140000C0140001001400014014080
:1014300000180140001C0140080001400804014060
:10144000024693680B400BB1012000E0002070477A
:1014500010B5C26821EA020302EA010443EA044328
:10146000036110BD0AB1016101E00B040361704723
:1014700001480068704700001C0000200348006815
:101480000349097808440149086070471C0000209E
:101490002400002010B50848006840F010000649FC
:1014A0000860032000F080F80F2000F007F800F03B
:1014B0002BF8002010BD00000020024070B504464B
:1014C0000E4800784FF47A71B1FBF0F00C490968CE
:1014D000B1FBF0F5284600F0F3FB08B1012070BD28
:1014E000102C07D200222146501E00F01EF805489D
:1014F000046001E00120F2E70020F0E72400002072
:101500000C000020200000207047014608460028FB
:1015100009DB00F01F0301229A4043099B0003F1FD
:10152000E023C3F8002100BF70472DE9F05F80463B
:101530000D461646002702F0E7F9074639462A46C7
:10154000334601F00700C0F1070ABAF1040F02D9CF
:101550004FF0040A01E0C0F1070AD14600F1040A85
:10156000BAF1070F02D24FF0000A01E0A0F1030A1E
:10157000D4464FF0010A0AFA09FAAAF1010A0AEA66
:10158000020A0AFA0CFA4FF0010B0BFA0CFBABF152
:10159000010B0BEA030B4AEA0B042146404602F01A
:1015A000BBF9BDE8F09F000000BF00F00702064B4A
:1015B00019684FF6FF031940044B0B4343EA02211D
:1015C000014B196000BF70470CED00E00000FA0508
:1015D00000BF00BF00BF00BF00BFBFF34F8F00BF01
:1015E00000BF00BF0948006800F4E06008490843F4
:1015F000001D0649086000BF00BF00BFBFF34F8F4A
:1016000000BF00BF00BF00BF00BFFDE70CED00E062
:101610000000FA0570B504460D460CB9012070BDF6
:101620005A48006800F00700A8420ED257480068E8
:1016300020F007002843554908600846006800F07C
:101640000700A84201D00120E9E7207800F002005D
:1016500002281DD1207800F00400042805D14C4850
:10166000406840F4E0604A494860207800F0080093
:10167000082805D14648406840F460504449486015
:101680004348406820F0F000A168084340494860A2
:10169000207800F0010078B36068012806D13C484A
:1016A000006800F4003090B90120B8E760680228B3
:1016B00006D13748006800F0007040B90120AEE75D
:1016C0003348006800F0020008B90120A7E730485D
:1016D000406820F00300616808432D494860FFF727
:1016E000C7FE064609E0FFF7C3FE801B41F28831C2
:1016F000884202D9032092E707E02548406800F0BD
:101700000C006168B0EB810FEDD12048006800F05B
:101710000700A8420ED91D48006820F007002843A2
:101720001A4908600846006800F00700A84201D086
:10173000012074E7207800F00400042807D1144841
:10174000406820F4E060E16808431149486020786F
:1017500000F00800082808D10D48406820F46050C7
:10176000216940EAC1000A49486000F03FF8084991
:101770004968C1F30311074A515CC8400649086033
:1017800006480068FFF79AFE002048E70020024064
:1017900000100240C83E00080C000020200000207D
:1017A00001480068704700000C00002000B5FFF7FA
:1017B000F7FF04494968C1F30221034A515CC8405C
:1017C00000BD000000100240D83E000800B5FFF741
:1017D000E7FF04494968C1F3C221034A515CC8408C
:1017E00000BD000000100240D83E000870B5002186
:1017F0000022002400230020134D696801F00C052D
:10180000F5B1042D02D0082D19D101E00F4819E0DF
:101810000F4DC1F38346AB5D01F4803555B10A4DE0
:101820006D68C5F340450B4E725D084D5D43B5FBD9
:10183000F2F402E0084D03FB05F4204602E000BF8D
:10184000024800BF00BF70BD0010024000127A00C5
:10185000E03E0008F03E000800093D00F8B50446EF
:101860000CB90120F8BD207800F00100002878D0E4
:10187000F848406800F00C0004280CD0F548406897
:1018800000F00C00082811D1F248406800F48030C4
:10189000B0F5803F0AD1EF48006800F4003000281E
:1018A0005FD0606800285CD10120DBE700BF606882
:1018B000B0F5803F06D1E748006840F48030E54944
:1018C000086028E0606858B9E248006820F4803079
:1018D000E04908600846006820F4802008601AE0AB
:1018E0006068B0F5A02F0BD1DA48006840F4802082
:1018F000D84908600846006840F4803008600AE073
:10190000D448006820F48030D24908600846006856
:1019100020F48020086000BF606888B1FFF7A8FD50
:10192000054606E0FFF7A4FD401B642801D903200B
:1019300098E7C848006800F400300028F2D010E0B2
:10194000FFF796FD054606E0FFF792FD401B642871
:1019500001D9032086E7BF48006800F40030002862
:10196000F2D1207800F00200022857D1B94840682F
:1019700000F00C0050B1B748406800F00C00082897
:1019800018D1B448406800F4803098B9B148006874
:1019900000F0020020B12069012801D0012061E798
:1019A000AC48006820F0F800616940EAC100A9492C
:1019B000086033E02069E8B10120A7490860FFF71B
:1019C00057FD054606E0FFF753FD401B022801D9ED
:1019D000032047E79F48006800F002000028F2D08B
:1019E0009C48006820F0F800616940EAC10099490C
:1019F000086013E0002098490860FFF739FD0546AC
:101A000006E0FFF735FD401B022801D9032029E736
:101A10009048006800F002000028F2D1207800F021
:101A2000080008282DD1A069B8B101208B490860B1
:101A3000FFF71EFD054606E0FFF71AFD401B0228D2
:101A400001D903200EE78348406A00F00200002815
:101A5000F2D0012001F0CCF813E000207F490860AB
:101A6000FFF706FD054606E0FFF702FD401B0228D2
:101A700001D90320F6E67748406A00F0020000280A
:101A8000F2D1207800F00400042873D100277148B7
:101A9000C06900F0805070B900BF6E48C06940F066
:101AA00080506C49C8610846C06900F080500090C1
:101AB00000BF00BF01276A48006800F48070B0B919
:101AC0006748006840F4807065490860FFF7D0FC03
:101AD000054606E0FFF7CCFC401B642801D9032033
:101AE000C0E65F48006800F480700028F2D000BFB4
:101AF000E068012806D15748006A40F001005549C6
:101B0000086227E0E06858B95248006A20F00100F6
:101B1000504908620846006A20F00400086219E093
:101B2000E06805280BD14B48006A40F004004949A1
:101B300008620846006A40F0010008620AE0454871
:101B4000006A20F00100434908620846006A20F05C
:101B50000400086200BFE068A0B1FFF789FC0546F9
:101B600009E0FFF785FC401B41F28831884202D929
:101B7000032077E622E03748006A00F002000028E0
:101B8000EFD012E0FFF774FC054608E0FFF770FCA9
:101B9000401B41F28831884201D9032062E62D487A
:101BA000006A00F002000028F0D1012F05D1294879
:101BB000C06920F080502749C86100BFE069C8B300
:101BC0002448406800F00C00082860D0E069022832
:101BD00048D1002020490866FFF74AFC054606E088
:101BE000FFF746FC401B022801D903203AE61948BA
:101BF000006800F000700028F2D1206AB0F5803F44
:101C000007D11448406820F40030A1680843114906
:101C10004860D4E9080108430E49496821F4741169
:101C200008430C49486001200B490866FFF720FC77
:101C3000054607E03DE0FFF71BFC401B022801D9E9
:101C400003200FE60348006800F000700028F2D07F
:101C50002FE0000000100240000042428004424297
:101C600000700040002014490866FFF701FC05469B
:101C700006E0FFF7FDFB401B022801D90320F1E538
:101C80000E48006800F000700028F2D111E0E06911
:101C9000012800D1E6E50948466806F48031206A4B
:101CA000814204D106F47011606A814201D00120A2
:101CB000D8E50020D6E500000000424200100240B6
:101CC00070B504462546681EB0F1807F01D301201F
:101CD0000FE0681E4FF0E02148610F214FF0FF3008
:101CE00001F01AFE00204FF0E02188610720086112
:101CF000002070BD10B504460CB9012010BD94F849
:101D00003D0028B9002084F83C00204600F025F86A
:101D1000022084F83D00211D206801F007FA01200F
:101D200084F8460000BF84F83E0001213F200155A1
:101D3000402001554120015500BF00BF012084F81B
:101D4000420043200155442001554520015500BF64
:101D5000012084F83D000020D0E77047014691F84B
:101D60003D00012801D001207047022081F83D008C
:101D70000868C06840F001000B68D860164B08681E
:101D8000984213D0154B086898420FD00868B0F1FC
:101D9000804F0BD0124B0868984207D0114B08684F
:101DA000984203D0104B086898420CD108688068AC
:101DB00000F00702062A0CD00868006840F0010015
:101DC0000B68186005E00868006840F001000B68C7
:101DD00018600020C8E70000002C014000340140DA
:101DE0000004004000080040000C0040F8B5044624
:101DF0000D46164694F8420020282DD105B10EB9A3
:101E00000120F8BD0120206300206063324629468E
:101E1000204601F0D5FB0746206B012819D100BFF1
:101E200000200090206800680090206840680090C2
:101E300000BF00BF00BF00BF21680C3151E8001F88
:101E400041F0100021680C3141E80002002AF3D172
:101E500000E001273846D4E70220D2E770B50446F7
:101E60000D4607492068884208D1012005490870BD
:101E700040F68842491C0448FFF7B8FF70BD0000D7
:101E80000044004044030020D80F002070470000A9
:101E90002DE9F84F0446206805682068C668206868
:101EA00047694FF00009CA4605F00F09B9F1000F64
:101EB0000AD105F0200038B106F0200020B12046FC
:101EC00001F081FABDE8F88FB9F1000F7BD007F07F
:101ED000010018B906F49070002874D005F00100D4
:101EE00030B106F4807018B1606C40F0010060649D
:101EF00005F0040030B107F0010018B1606C40F04B
:101F00000200606405F0020030B107F0010018B172
:101F1000606C40F00400606405F0080048B106F011
:101F2000200010B907F0010018B1606C40F0080003
:101F30006064606C002845D005F0200028B106F0F0
:101F4000200010B1204601F03EFA20684069C0F33D
:101F5000801A606C00F0080010B9BAF1000F2CD0A4
:101F6000204601F0D7F92068406900F0400000B336
:101F700000BF00BF2168143151E8001F21F040006C
:101F80002168143141E80002002AF3D100BFE06B60
:101F900050B17748E16B4863E06BFEF7ABFC88B16A
:101FA000E06B416B88470DE02046FFF76FFF09E0CB
:101FB00009E02046FFF76AFF04E02046FFF766FFCE
:101FC000002060647EE7206B012877D105F01000C7
:101FD000002873D006F010000028FAD000BF0020BF
:101FE000009020680068009020684068009000BF62
:101FF00000BF2068406900F0400000285FD0E06B1F
:10200000006840681FFA80F8B8F1000F55D0A08D25
:10201000404552DDA4F82E80E06B8069202843D033
:1020200000BF00BF21680C3151E8001F21F480700F
:1020300021680C3141E80002002AF3D100BF00BF43
:1020400000BF2168143151E8001F21F00100216810
:10205000143141E80002002AF3D100BF00BF00BFE5
:102060002168143151E8001F21F04000216814312B
:1020700041E80002002AF3D100BF202084F842008A
:102080000020206300BF00BF21680C3151E8001F11
:1020900021F0100021680C3141E80002002AF3D140
:1020A00000BFE06BFEF7FAFB02206063A08DE28DBB
:1020B000801A81B22046FFF7D1FE03E742E0A08DEF
:1020C000E18D401A1FFA80F8E08DD0B3B8F1000F0F
:1020D00037D000BF00BF21680C3151E8001F21F448
:1020E000907021680C3141E80002002AF3D100BF52
:1020F00000BF00BF2168143151E8001F21F001002A
:102100002168143141E80002002AF3D100BF2020E9
:1021100084F842000020206300BF00BF21680C311A
:1021200051E8001F21F0100021680C3141E8000245
:10213000002AF3D100BF0220606341462046FFF72A
:102140008DFEBFE605F0800030B106F0800018B1CA
:10215000204601F0B9FAB5E605F0400030B106F0CE
:10216000400018B1204601F00BF9ABE600BFA9E62C
:10217000D931000810B504460CB9012010BDA06982
:1021800000B100E000BF94F8410028B9002084F8B5
:102190004000204600F02AF8242084F841002068FE
:1021A000C06820F400502168C860204601F08AF918
:1021B0002068006920F49040216808612068406927
:1021C00020F02A00216848612068C06840F400506F
:1021D0002168C86000206064202084F8410084F8F1
:1021E00042000020606300BFC8E7000010B586B061
:1021F00004462849206888424AD100BF00BF2648CB
:10220000806940F00400244988610846806900F034
:102210000400019000BF00BF00BF00BF00BF084620
:10222000806940F0040088610846806900F004007D
:10223000019000BF00BF00BF00BF00BF084680691B
:1022400040F4804088610846806900F48040019035
:1022500000BF00BF00BF481502900220039001207C
:1022600004900320059002A90C48FEF749FF4FF4A3
:10227000806002900020039002A90848FEF740FF0A
:102280002520FFF742F9032211462520FFF74DF9DB
:1022900006B010BD003801400010024000080140A7
:1022A00070B504460D46164694F8420020280BD11E
:1022B00005B10EB9012070BD0020206332462946C9
:1022C000204601F0E1F9F6E70220F4E710B50446F4
:1022D0002049206888423BD11F48008800F4004014
:1022E00088BB1D48008800F4804070B11B4800780E
:1022F0000A2803D000201849088024E016480088E6
:1023000040F40040144908801DE0144800780D286E
:1023100006D11148008840F480400F49088012E03F
:102320000E4800780C490988C1F30D010C4A50543D
:1023300009480088401C0849088008460088C728CA
:1023400001DD00200880012204490648FFF7A8FFAC
:1023500010BD000000380140180000201A000020C5
:10236000540000201C01002070472DE9F84F04465E
:102370000E46174699464FF0000A94F8410020286F
:1023800050D106B117B90120BDE8F88F0020606474
:10239000212084F84100FFF76BF88246A784E78488
:1023A000A068B0F5805F04D1206910B90025B0465F
:1023B00002E035464FF000081EE05346002280211F
:1023C0002046CDF8009001F0AFF920B1202084F82C
:1023D00041000320D8E745B9B8F80000C0F3080071
:1023E0002168486008F1020803E028782168486005
:1023F0006D1CE08C401EE084E08C0028DDD153464B
:10240000002240212046CDF8009001F08DF920B146
:10241000202084F841000320B6E7202084F8410002
:102420000020B1E70220AFE7704700BFFEE70000E1
:1024300008B5434A811A904241D009DC4149014420
:1024400081B1B1F5806F1CD0B1F5006F74D127E078
:10245000B1F5806F42D0B1F5006F4ED0B1F5406F4D
:102460006AD159E000BF3849896941F00401364A10
:1024700091611146896901F00401009100BF00BF1C
:102480005BE000BF3049896941F008012E4A916143
:102490001146896901F00801009100BF00BF4CE0BE
:1024A00000BF2949896941F01001274A916111460D
:1024B000896901F01001009100BF00BF3DE000BF3D
:1024C0002149896941F020011F4A916111468969BA
:1024D00001F02001009100BF00BF2EE000BF1A49AB
:1024E000896941F04001184A91611146896901F0FA
:1024F0004001009100BF00BF1FE000BF1249896981
:1025000041F08001104A91611146896901F0800112
:10251000009100BF00BF10E000BF0B49896941F482
:102520008071094A91611146896901F480710091B5
:1025300000BF00BF01E0FFE700BF00BF08BD000013
:102540000014014000F8FEBF0010024070B50446C0
:10255000002500267CB180220021084601F096FC6F
:1025600080220121002001F091FC80220321002023
:1025700001F08CFC0EE000221146104601F086FCB2
:1025800000220121104601F081FC002203211046A7
:1025900001F07CFC70BD000010B507480068401CCD
:1025A00005490860084600680F2804D30F2008601A
:1025B0000020FFF7CBFF10BD0800002010B586B04B
:1025C00000BF2F48806940F001002D49886108460E
:1025D000806900F00100019000BF00BF00BF2949E1
:1025E000486820F0E06040F00070486000BF0020C4
:1025F000029003900490059000243DE004EB440118
:10260000214A02EB81014868FFF712FF04EB440006
:102610001D4931F82000029000200390049003200F
:10262000059004EB4401184A02EB8101486802A9B5
:10263000FEF766FD04EB440101EBC401134A02EB13
:10264000810023460022124901F0D6FA04EB44012E
:1026500001EBC4010D4A02EB81000E4A032101F097
:1026600071F904EB440101EBC401084A02EB81005B
:1026700001F0FEFA601CC4B2082CBFD306B010BD36
:10268000001002400000014004520008E401002054
:10269000493C00085939000810B50446FDF7E0FE32
:1026A0000120FFF753FF0020024908600248047030
:1026B00010BD00000800002005000020014908604E
:1026C000704700002800002000B585B000BF1A4800
:1026D000806940F00800184988610846806900F068
:1026E0000800009000BF00BF00BF0846806940F0AE
:1026F000400088610846806900F04000009000BFFB
:1027000000BF47F601400190012002900390032092
:10271000049001A90948FEF7F3FC4FF47F400190B3
:102720000120029003900320049001A90448FEF7C1
:10273000E7FC05B000BD000000100240000C0140A5
:102740000018014010B5E92001F074F82B2001F0C9
:1027500071F8242001F06EF8812001F06BF8BE20A2
:1027600001F068F8A42001F065F8A62001F062F8F5
:10277000C02001F05FF8A32001F05CF8D12001F047
:1027800059F8D52001F056F8DA2001F053F8F4207A
:1027900001F050F8252001F04DF8F62001F04AF83C
:1027A0005A2001F047F8F52001F044F8002001F02C
:1027B00041F8F72001F03EF89F2001F03BF8F820A7
:1027C00001F038F8892001F035F8AD2001F032F839
:1027D000402001F02FF8502001F02CF8C42001F027
:1027E00029F8902001F026F8FF2001F023F884203A
:1027F00001F020F8F12001F01DF89F2001F01AF8F7
:1028000010BD000010B500BF012291020E48FEF776
:1028100029FE00BF0A2001F059FA00BF00224FF440
:1028200080610948FEF71EFE00BF022001F04EFA4B
:1028300000BF012291020448FEF714FE00BF96205B
:1028400001F044FA10BD0000000C014008B5434AF5
:10285000811A904241D009DC4149014481B1B1F56E
:10286000806F1CD0B1F5006F74D127E0B1F5806F97
:1028700042D0B1F5006F4ED0B1F5406F6AD159E04A
:1028800000BF3849896941F00401364A9161114617
:10289000896901F00401009100BF00BF5BE000BF47
:1028A0003049896941F008012E4A916111468969D0
:1028B00001F00801009100BF00BF4CE000BF2949B2
:1028C000896941F01001274A91611146896901F037
:1028D0001001009100BF00BF3DE000BF21498969A0
:1028E00041F020011F4A91611146896901F02001E0
:1028F000009100BF00BF2EE000BF1A49896941F076
:102900004001184A91611146896901F04001009126
:1029100000BF00BF1FE000BF1249896941F080017C
:10292000104A91611146896901F08001009100BF50
:1029300000BF10E000BF0B49896941F48071094A6A
:1029400091611146896901F48071009100BF00BF57
:1029500001E0FFE700BF00BF08BD00000014014018
:1029600000F8FEBF001002401FB5002447E02749D1
:1029700001EB04110868FFF769FF244800EB04101D
:102980008088009001200190204800EB04108068AE
:1029900003901E4800EB0410C06802901B4901EB35
:1029A000041108686946FEF7ABFB184B03EB0413F0
:1029B000DA79164B03EB04139988144B03EB0413D9
:1029C0001868FEF74FFD114800EB0410807950B9EC
:1029D0000E4800EB0410C07908B9012000E0002087
:1029E0000B49085509E0094800EB0410C07901289B
:1029F00000D100E0002006490855601CC4B2142C28
:102A0000B5DB0121002000F06FF81FBDF43E000887
:102A10008801002070B50446142C00DB70BD0C4802
:102A200000EB0410807908B9012500E00025084A70
:102A300002EB04129188064A02EB041210682A463F
:102A4000FEF710FD00200349085500BFE6E700002F
:102A5000F43E00088801002070B50446142C00DB09
:102A600070BD0C4800EB0410807908B9002500E027
:102A70000125084A02EB04129188064A02EB04126F
:102A800010682A46FEF7EEFC01200349085500BFF6
:102A9000E6E70000F43E0008880100202DE9F0413F
:102AA0000446E0780006A17840EA0140617840EAF7
:102AB0000120217840EA010600250121002000F0D4
:102AC00013F801250CE00120A840304008B1012096
:102AD00000E000200746E8B2394600F005F86D1C1A
:102AE000142DF0D3BDE8F08170B505460C46012CDD
:102AF00003D12846FFF7B0FF02E02846FFF78AFF20
:102B000070BD000010B50446142C00DB10BD0A4A4D
:102B100002EB04129188084A02EB04121068FEF7D7
:102B200097FC0648005D012801D0012000E000204C
:102B30000249085500BFE9E7F43E0008880100207B
:102B400010B5044AD2F8841CD2F8800CFDF718FDA9
:102B500010BD0000A810002010B5FFF7B5FD00BFA4
:102B6000012211460548FEF77DFC00BFFFF74AFE33
:102B7000FFF7E8FDFDF7BEFC10BD0000000C0140B2
:102B800000BFFEE710B5FDF729FCFFF7D9FF4FF4B2
:102B9000FA7001F09BF84FF4FA7001F097F84FF4D7
:102BA000FA7001F093F84FF4FA7001F08FF810BD4D
:102BB00000BFFEE77047000006480078401C05494A
:102BC00008700846007918B108464079401C4871E1
:102BD0007047000038000020002004498871087107
:102BE0004871C871012048807047000038000020FB
:102BF00008B508490968C9084FF47A72B1FBF2F1C7
:102C00004143009100BF00BF00994A1E0092002975
:102C1000F9D108BD0C00002000B585B000BF00BF91
:102C20005348806940F00400514988610846806932
:102C300000F00400009000BF00BF00BF00BF00BF55
:102C40000846806940F0040088610846806900F009
:102C50000400009000BF00BF00BF00BF00BF0846D7
:102C6000806940F0040088610846806900F0040033
:102C7000009000BF00BF00BF00BF00BF0846C06992
:102C800040F40030C8610846C06900F4003000908C
:102C900000BF00BF00BF002001900290039004908D
:102CA0000420019002200290012003900320049050
:102CB00001A93048FEF724FA082001900020029074
:102CC00001A92C48FEF71CFA022001900120029075
:102CD00001A92848FEF714FA27482849086000206F
:102CE00048600021254881608021C1600021016188
:102CF000416181614FF44051C161FEF79BF800BF13
:102D00001E481F49C86308461C49486200BF10207E
:102D1000FEF7FBFB002211461020FEF706FC1948C7
:102D20001749086018484860002115488160C16053
:102D3000016181610C2141610021C161FFF71AFA33
:102D40002620FEF7E2FB002201212620FEF7EDFB04
:102D500000BF012202210748FEF784FB00BF40F6B6
:102D600088420A490648FFF741F805B000BD000057
:102D700000100240000801406C00024020100020BA
:102D8000D80F00200044004060AE0A004503002038
:102D900070B504460D462E462CB15D480078A04221
:102DA00001D05B4804705B480078002876D0002092
:102DB00058490870012640F688415648401CFDF7E6
:102DC00081FB012854D10020534908604FF4486228
:102DD0005049491C5148FDF72DFA514951480268A4
:102DE0000A604068486008460079892834D108465E
:102DF0004079452830D14FF4486248494A48FDF7A8
:102E00005EFA474840784649097840EA0120464939
:102E1000C1F8800C4248C0784149897840EA0120D5
:102E20004149C1F8840CFDF7F3FAFDF719FBFDF7F2
:102E300061FBFFF785FE4FF4FA7000F047FF4FF497
:102E4000FA7000F043FF4FF4FA7000F03FFF4FF4C8
:102E5000FA7000F03BFF19E034492E48D0F8810C9D
:102E600008600846FFF71AFE2C4800F0BDF80DE098
:102E700029480068401C2849086008460068032863
:102E800004D3FFF7C9FE0020234908600020284929
:102E9000887108714871C8710120488024484088B1
:102EA00010B923488079B0B11948007838B1184872
:102EB0000178002000F082F80020154908701C48B5
:102EC0000078372807DD12480178012000F076F8F5
:102ED00000200F49087016484079282808DD012095
:102EE00013498871002048710846C079401CC87198
:102EF0000F48C079052808DB002605200C49C87159
:102F0000FFF78AFE01200A494880304670BD000064
:102F1000400000204403002050000020301D00200D
:102F200045000020C50F0020A8100020410000200F
:102F3000380000202DE9FC4104460D4616460027C6
:102F400001208DF800008DF801408DF802508DF8B9
:102F5000036004216846FDF795FA074638128DF89C
:102F60000400F8B28DF805000621684600F008F864
:102F7000002002494880BDE8FC81000038000020A4
:102F800070B504460D4600BF002202210948FEF735
:102F900069FA00BFAAB24FF47A7321460648FFF7D8
:102FA000E4F900BF012202210248FEF75BFA00BFEC
:102FB00070BD000000080140D80F002070B5044625
:102FC0000D462A4621460320FFF7B4FF002004499E
:102FD00048800870012008710020487170BD000011
:102FE0003800002070470000F8B5064600BFD52025
:102FF00000F020FC00BF21A00068009000210846DE
:1030000000F03EF8002436E000252DE004EB8401BA
:1030100005EB8101715C6A4602EB9111087800F0C2
:103020003FFC04EB840105EB8101715CC1F30111EC
:103030001DF8010000F034FC04EB840105EB810174
:10304000715CC1F381011DF8010000F029FC04EB63
:10305000840105EB8101715C01F003011DF80100A1
:1030600000F01EFC681C85B2142DCFDB002000F0A0
:1030700017FC601C84B2A02CC6DBF8BD000FF0FF6B
:1030800070B504460D4604F12500C4B204F00F00EB
:1030900000F0D0FBC4F3021141F0100000F0CAFBB5
:1030A00005F00F0141F0600000F0C4FB702141EA1F
:1030B000151000F0BFFB70BD10B5FEF7DFF910BDB5
:1030C0007047000010B515480068006900F0010065
:1030D00010B313480068401C114908600846006896
:1030E000C821B0FBF1F201FB120010B901200D491B
:1030F000087000F0D7FD00BF01210B48FEF7A8F9CA
:1031000000BFFDF791F9FFF757FDFFF745FA6FF0A4
:10311000010002490968086110BD00009C010020FF
:1031200000000020040000200008014010B50268E3
:10313000244B98420ED0244B98420BD0B0F1804FD4
:1031400008D0224B984205D0214B984202D0214B07
:10315000984203D122F070024B681A43194B9842EF
:103160000ED0194B98420BD0B0F1804F08D0174BBE
:10317000984205D0164B984202D0164B984203D184
:1031800022F44072CB681A4322F080034C6943EA70
:10319000040202608B68C3620B688362094B984229
:1031A00002D0094B984201D10B69036301234361AB
:1031B000036903F001031BB1036923F001030361F9
:1031C00010BD0000002C014000340140000400400C
:1031D00000080040000C004070B505466C6A0020F5
:1031E000E085E0842046FEF751FE70BD70B50646CE
:1031F0000025746A20684069C0F3C01594F8410046
:10320000212805D125B10020E084204600F0C8F82F
:1032100020684069C0F3801594F84200222805D147
:1032200025B10020E085204600F074F8606C40F085
:10323000100060642046FEF729FE70BD70B505469B
:103240006C6A2868006800F02000002842D1E08500
:1032500000BF00BF21680C3151E8001F21F48070CD
:1032600021680C3141E80002002AF3D100BF00BF01
:1032700000BF2168143151E8001F21F001002168CE
:10328000143141E80002002AF3D100BF00BF00BFA3
:103290002168143151E8001F21F0400021681431E9
:1032A00041E80002002AF3D100BF202084F8420048
:1032B000206B01280ED100BF00BF21680C3151E8FE
:1032C000001F21F0100021680C3141E80002002AA3
:1032D000F3D100BF00206063206B012804D1A18DD1
:1032E0002046FEF7BBFD02E02046FEF7EFFF70BD73
:1032F00070B505466C6A01206063206B012805D11A
:10330000A08D41082046FEF7A9FD02E02046FFF708
:103310002BF870BD00BF00BF02680C3252E8002FCE
:1033200022F4907102680C3242E80013002BF3D1B2
:1033300000BF00BF00BF0268143252E8002F22F025
:1033400001010268143242E80013002BF3D100BFE0
:10335000016B01290ED100BF00BF02680C3252E898
:10336000002F22F0100102680C3242E80013002BFB
:10337000F3D100BF202180F8421000210163704783
:1033800010B504462068C06820F040002168C8607D
:10339000202084F841002046FFF746F8002010BDA9
:1033A00000BF00BF02680C3252E8002F22F0C001BB
:1033B00002680C3242E80013002BF3D100BF202139
:1033C00080F841107047F8B5044694F8420022286E
:1033D00075D1A068B0F5805F0CD1206950B9002587
:1033E000A66A20684068C0F308003080A06A801C8C
:1033F000A06215E0A56A0026A068B0F5805F03D042
:10340000A06828B9206918B920684068287004E0CD
:103410002068406800F07F002870A06A401CA0620D
:10342000E08D401E80B2E085002846D12068C0684B
:1034300020F020002168C8602068C06820F48070F7
:103440002168C8602068406920F001002168486157
:10345000202084F8420000206063206B012826D1E0
:103460000020206300BF00BF21680C3151E8001F1D
:1034700021F0100021680C3141E80002002AF3D14C
:1034800000BF2068006800F0100010280AD100BFBB
:10349000002000902068006800902068406800903C
:1034A00000BF00BFA18D2046FEF7D8FC02E02046F9
:1034B000FEF70CFF0020F8BD01E00020FBE7022032
:1034C000F9E7000070B504462168096921F440510C
:1034D000E2681143226811612269A168114362699F
:1034E00041EA02052168C96841F20C62914329430F
:1034F0002268D1602168496921F44071A2691143B1
:10350000226851612D4A2168914202D1FEF75EF98D
:1035100001E0FEF74BF900EBC00101EB001162681E
:103520009200B1FBF2F100EBC00202EB0012636803
:103530009B00B2FBF3F26423B2FBF3F202EBC20393
:1035400003EB0212A1EB8201322202EB0111642291
:10355000B1FBF2F101F0F00100EBC00202EB00124E
:1035600063689B00B2FBF3F26423B2FBF3F201EB5E
:10357000021200EBC00101EB001163689B00B1FB7C
:10358000F3F100EBC00303EB00136668B600B3FB76
:10359000F6F36426B3FBF6F303EBC30606EB031363
:1035A000A1EB8301322303EB01116423B1FBF3F19F
:1035B00001F00F0111442268916070BD0038014094
:1035C00077B581B0044615460298A062A585002013
:1035D0006064222084F842002848E16B8862284811
:1035E000E16BC8622748E16B08630020E16B486328
:1035F00002AE32682368191D2B46E06BFDF760FCB4
:1036000000BF00200090206800680090206840689B
:10361000009000BF00BF206970B100BF00BF2168EB
:103620000C3151E8001F41F4807021680C3141E8F1
:103630000002002AF3D100BF00BF00BF216814318F
:1036400051E8001F41F001002168143141E80002F7
:10365000002AF3D100BF00BF00BF2168143151E838
:10366000001F41F040002168143141E80002002AA7
:10367000F3D100BF002004B070BD00003D3200084F
:10368000F1320008ED31000810B5034699629A85C1
:10369000DA8500205864222083F84200186928B196
:1036A0001868C06840F480701C68E0601868406961
:1036B00040F001001C6860611868C06840F020009C
:1036C0001C68E060002010BD014691F841002128EF
:1036D00028D18868B0F5805F0BD1086948B90A6ABB
:1036E0001088C0F308000B685860086A801C0862E4
:1036F00005E00B6A581C086218780B685860C88C83
:10370000401E80B2C88458B90868C06820F08000A4
:103710000B68D8600868C06840F040000B68D8604B
:10372000002070470220FCE72DE9F84304460D46CF
:1037300017469846089E31E0701C70B3FDF798FE5E
:10374000A0EB0800B04200D816B90320BDE8F8830A
:103750002068C06800F00400F8B1802D1ED0402D14
:103760001CD020680068C0F3C000B0B100BF0020CA
:10377000009020680068009020684068009000BFBA
:1037800000BF2046FFF7C6FD0820606400BF002090
:1037900084F8400000BF0120D8E7FFE720680068F8
:1037A0002840A84201D1012000E00020B842C3D047
:1037B0000020CBE70021044A1268D1B241EA00227E
:1037C000014B1A60704700000C18014010B5024808
:1037D000FEF75EFB10BD00001C01002010B5024882
:1037E000FEF756FB10BD0000D80F002000BFFEE71B
:1037F00000B585B000BF00BF0C48806940F00400F0
:103800000A4988610846806900F00400009000BF02
:1038100000BF00BF0120019002900390032004909C
:1038200001A90348FDF76CFC05B000BD0010024083
:103830000008014010B5044600BF00224FF480414B
:103840001648FDF70FFE00BF00BF01221103134809
:10385000FDF708FE00BF2046FFF7ACFF00BF0022C7
:103860004FF400610D48FDF7FDFD00BF00BF0022D1
:103870004FF400510948FDF7F5FD00BF00BF0122DC
:1038800051030648FDF7EEFD00BF00BF0122D10243
:103890000248FDF7E7FD00BF10BD0000000C01402D
:1038A00010B5044600BF012291031648FDF7DAFD6A
:1038B00000BF00BF012211031248FDF7D3FD00BF76
:1038C0002046FFF777FF00BF00224FF400610D484C
:1038D000FDF7C8FD00BF00BF00224FF400510948AA
:1038E000FDF7C0FD00BF00BF012251030548FDF7F1
:1038F000B9FD00BF00BF0122D1020248FDF7B2FDB1
:1039000000BF10BD000C014002480068C0F3022057
:10391000704700000CED00E010B5002804DB0A073A
:10392000130E054A135406E00A07140E034A00F06A
:103930000F031B1FD45410BD00E400E018ED00E09D
:1039400000BF704708B1072900DB704700F10C0386
:1039500043F8212000BFF8E770B504467CB1084861
:10396000006860B12579082D08D205EB4501054AAC
:1039700002EB8101087A02490968884700BF70BDDF
:10398000280000200452000870B5044600BF2079CA
:10399000A16888470546E07800F00700002802DDAE
:1039A0002088401C2080E078B5EBD01F13D0E07851
:1039B000C008401CE17860F3C501E170C1F3C200AA
:1039C00003280CDBE07865F3C710E070E07820F0A6
:1039D0003800E07003E0E07820F03800E070E07834
:1039E00000F0070005287DD2DFE800F0032858AF7B
:1039F000DB00E078C0F38010E178B0EBD11F17D185
:103A0000A07820F0F000A07000BFE06810B1204660
:103A1000E168884700BF00202080A07820F00F00D8
:103A2000401CA070E07820F00700401CE07004E02B
:103A3000A07820F0F0008030A070DBE0E078C0F3E8
:103A40008010E178B0EBD11F13D0A07820F0F00007
:103A50001030A07000BF206910B12046216988474E
:103A600000BF00202080E07820F00700801CE0707C
:103A700013E02088C82810DDA07820F0F000503036
:103A8000A07000BF206A10B12046216A884700BF9D
:103A9000E07820F00700001DE070ABE0E078C0F3B4
:103AA0008010E178B0EBD11F25D1A07820F0F00094
:103AB000A07000BFE06810B12046E168884700BFF1
:103AC000A07800F00F000F2804DAA078411C61F301
:103AD0000300A07000BF606910B12046616988478B
:103AE00000BF00E081E000202080E07820F00700A7
:103AF000C01CE07028E020883C2825DDA07800F07C
:103B00000F0001280BD1A07820F0F0003030A07019
:103B100000BFA06910B12046A169884710E0A078D5
:103B200000F00F0002280BD1A07820F0F000403008
:103B3000A07000BFE06910B12046E169884700BF6E
:103B4000E07820F00700E07054E0E078C0F38010E7
:103B5000E178B0EBD11F1BD0A07820F0F00010303E
:103B6000A07000BF206910B120462169884700BFBE
:103B700020883C2807DA00202080E07820F0070029
:103B8000801CE0700CE0E07820F00700E07007E0B7
:103B900020883C2804DDE07820F00700401CE0701D
:103BA00028E0E078C0F38010E178B0EBD11F0BD1B2
:103BB000A07820F0F0006030A07000BF606A10B103
:103BC0002046616A88470FE0A07820F0F0001030AE
:103BD000A07000BF206910B120462169884700BF4E
:103BE000E07820F00700E07004E0E07820F00700C3
:103BF000E07000BF00BF70BD2DE9F04104460D46E6
:103C000016461F4604B10DB9BDE8F0812C212046AF
:103C1000FCF787FBA07820F0F0008030A070A56052
:103C20000EB9012000E00020E17860F3C711E170D7
:103C3000E07866F38610E0702771E07820F00700E6
:103C4000E07000BFE0E7000070B5044604EB4402FA
:103C5000064B33F8221004EB440203EB8202506857
:103C6000FDF7EEFB0546284670BD00000452000833
:103C7000014611B96FF0010070470948026805E07C
:103C80008A4202D14FF0FF30F6E7926A002AF7D15C
:103C9000034800688862024801600020ECE70000E9
:103CA0003400002010B50548046803E02046FFF703
:103CB0006BFEA46A002CF9D110BD00003400002076
:103CC00001490860704700001000002010B504464C
:103CD0004FF47A7104FB01F000F002F810BD00000F
:103CE00070B5034600224FF0E02675690D4E366828
:103CF00003FB06F44FF0E026B16910E04FF0E02638
:103D0000B06988420BD0884202D20E1A324402E0D7
:103D10002E1A0E4432440146A24200D300E0EDE7E1
:103D200000BF70BD1000002038B504460D4600BF2E
:103D300000BF1248C06940F001001049C861084640
:103D4000C06900F00100009000BF00BF00BF880400
:103D50000B4908600846456000218160C460FDF79A
:103D6000C9FF002202211C20FDF7DFFB1C20FDF70C
:103D7000CCFB0348FDF7F2FF38BD00000010024005
:103D80009C010020FDF786FB4FF4E01000F04AF89C
:103D90004820FFF795FFFEF7E7FDFEF70FFCFFF762
:103DA00027FDFEF739FFFEF7D7FEFEF715FFFEF7FA
:103DB000E9FE41F61F413120FFF7B6FF1348FEF739
:103DC0007DFC22E012480078012809D111480078D2
:103DD000012805D100200F4908700120FEF792FE4E
:103DE0000B4801780C480078FEF7D2FF08490870AC
:103DF000002009490870094800680949884204D927
:103E0000FDF7E6FB002005490860DBE7992600087E
:103E10000600002004000020050000200000002013
:103E200040420F0030B58FB005460124282105A877
:103E3000FCF777FA14216846FCF773FA0120059025
:103E4000000406900020079002200C90C1030D9101
:103E50000E9505A8FDF702FD04460CB100BFFEE774
:103E60000F20009002200190002002904FF480600B
:103E700003900020049002216846FDF7CBFB044626
:103E80000CB100BFFEE70FB030BD0000F8B505462D
:103E90000E4614460BA00068009031462846FFF7F6
:103EA000EFF8694601EB94110878FFF7F9FCC4F3C9
:103EB00040121DF81200FFF7F3FC9DF80000FFF719
:103EC000EFFCF8BD000FF0FF000000000000000054
:103ED00001020304060708090000000001020304B0
:103EE00002030405060708090A0B0C0D0E0F10103B
:103EF0000102000000100140000100010300000069
:103F00000100000000100140000200010300000059
:103F10000100000000080140000200010300000051
:103F2000010000000008014000080001030000003B
:103F300001000000000801400080000103000000B3
:103F40000100000000100140000800010300000013
:103F50000100000000140140010000010300000006
:103F600001000000001401400400000103000000F3
:103F700001000000001401401000000103000000D7
:103F80000100000000140140400000010300000097
:103F9000010000000010014080000001030000004B
:103FA00001000000000801400001000103000000C2
:103FB00001000000000801400004000103000000AF
:103FC0000100000000080140001000010300000093
:103FD0000100000000100140000400010300000087
:103FE000010000000010014000100001030000006B
:103FF0000100000000140140020000010300000065
:10400000010000000014014008000001030000004E
:104010000100000000140140200000010300000026
:1040200001000000001401408000000103000000B6
:10403000010000000000000000000000000000007F
:1040400000002020202020200020000000285050C8
:10405000000000000000000000002828FC2850FCA0
:1040600050500000002078A8A0603028A8F0200060
:10407000000048A8B05028345448000000002050E8
:104080005078A8A8906C000000404080000000001C
:1040900000000000000408101010101010080400A8
:1040A00000402010101010101020400000000020D0
:1040B000A87070A8200000000000202020F8202018
:1040C00020000000000000000000000000404080D0
:1040D0000000000000F800000000000000000000E8
:1040E0000000000060600000000810101020204058
:1040F00040408000000070888888888888700000B0
:104100000000206020202020207000000000708827
:104110008810204080F800000000708808300808EF
:104120008870000000001030505090781018000087
:104130000000F88080F0080888700000000070908F
:1041400080F08888887000000000F89010202020FF
:104150002020000000007088887088888870000027
:1041600000007088888878084870000000000060AF
:1041700060000000006060000000000000200000FF
:104180000020200000040810204020100804000037
:1041900000000000F80000F80000000000402010BF
:1041A00008040810204000000000708888102020BB
:1041B000002000000000708898A8A8B8807800004F
:1041C000000020203050507848CC00000000F0481B
:1041D0004870484848F0000000007888808080805F
:1041E000887000000000F0484848484848F0000047
:1041F0000000F8485070504048F800000000F848AF
:104200005070504040E000000000384880809C889A
:10421000483000000000CC484878484848CC0000AE
:104220000000F8202020202020F8000000007C1052
:10423000101010101090E0000000EC48506050503A
:1042400048EC00000000E0404040404044FC0000DA
:104250000000D8D8D8D8A8A8A8A800000000DC483A
:104260006868585848E80000000070888888888886
:10427000887000000000F0484870404040E00000B6
:1042800000007088888888E8987018000000F0485E
:104290004870504848EC00000000788880601008A2
:1042A00088F000000000F8A82020202020700000E6
:1042B0000000CC4848484848483000000000CC483E
:1042C00048505030202000000000A8A8A87050508E
:1042D000505000000000D8505020205050D800000E
:1042E0000000D85050202020207000000000F890DE
:1042F0001020204048F800000038202020202020F6
:1043000020203800004040402020101010080000FD
:1043100000701010101010101010700000205000CD
:10432000000000000000000000000000000000008D
:10433000000000FC00200000000000000000000061
:104340000000000000304838483C00000000C04039
:1043500040704848487000000000000000384840A5
:10436000403800000000180808384848483C000061
:1043700000000000003048784038000000001C2099
:10438000207820202078000000000000003C483009
:10439000407844380000C0404070484848EC000075
:1043A00000002000006020202070000000001000AD
:1043B00000301010101010E00000C040405C507041
:1043C00048EC00000000E0202020202020F8000021
:1043D0000000000000F0A8A8A8A80000000000004D
:1043E00000F0484848EC0000000000000030484859
:1043F000483000000000000000F04848487040E0ED
:1044000000000000003848484838081C0000000040
:1044100000D8604040E0000000000000007840301C
:1044200008780000000000202070202020180000E4
:104430000000000000D84848483C00000000000090
:1044400000EC4850302000000000000000A8A870D8
:10445000505000000000000000D8502050D800004C
:104460000000000000EC4850302020C00000000098
:104470000078102020780000001810101020101074
:104480001010180010101010101010101010101034
:1044900000602020201020202020600040A4180070
:1044A000000000000000000000000000000000000C
:1044B0000000000000001010101010100018000084
:1044C0000012244800000000000000000000242426
:1044D000FE4848FE4848000000103C545030181474
:1044E000547810000000E4A4A8F01E2A2A4E000010
:1044F00000003048487EA494887700000060204087
:10450000000000000000000000020C081010101055
:104510000808060000402010080808081020400085
:1045200000000010927C7C9210000000000010102F
:1045300010FE10101000000000000000000000003D
:104540000060204000000000007F0000000000002C
:1045500000000000000000000060000000010206F2
:10456000040808102020400000003C24424242423F
:10457000243C00000000107010101010107C00008F
:1045800000003C4242040810627E000000003C42F1
:10459000021C0202423C000000000C142444443C73
:1045A000040C000000007E40407C0202423C0000FF
:1045B00000001C24405C6242623C000000007E441B
:1045C000080810101010000000003C4242342C4239
:1045D000423C00000000186442463A02243C0000BD
:1045E000000000001800000000180000000000009B
:1045F00000100000001010000002041820402010DD
:104600000C02000000000000FE0000FE00000000A0
:1046100000402018040204083040000000003C4222
:1046200062020C080018000000003C469AAAAABCCE
:10463000403E0000000010182824247C42E70000BF
:104640000000F8444478464242FC000000003E422C
:1046500080808080423C00000000F8444242424298
:1046600044F800000000FC424878484042FC00004A
:104670000000FC424878484040E0000000003C4414
:1046800080808E84443800000000E742427E42422F
:1046900042E7000000007C1010101010107C000099
:1046A00000003E08080808080888F0000000EE44F2
:1046B0004870504844EE00000000E0404040404058
:1046C00042FE00000000EE6C6C6C545454D60000A6
:1046D0000000C76252524A4646E2000000003C44D5
:1046E00082828282443800000000FC42427C4040CA
:1046F00040E0000000003844828282B24C3806005C
:104700000000FC42427C484446E3000000003E4278
:1047100040380402427C00000000FE92101010108D
:10472000103800000000E74242424242423C000092
:104730000000E74244242C28181000000000D69204
:1047400092929A6C644400000000E76624181824D2
:1047500066E700000000EE44283810101038000012
:1047600000007E840810102042FC0000001E101083
:104770001010101010101E0000402020101008080B
:1047800004040200007808080808080808087800EF
:10479000001C2200000000000000000000000000DB
:1047A00000000000000000FF0020000000000000EA
:1047B0000000000000000000003C423E423F0000BC
:1047C0000000C040405C6242427C000000000000EB
:1047D000003C6240423C000000000602021E6242B1
:1047E000423F000000000000003C427E403E0000CE
:1047F00000000F10107E1010107C00000000000060
:10480000003E4438407C423C0000C040405C624274
:1048100042E700000000300000701010107C000023
:1048200000000C00001C0404040404780000C040D4
:10483000404E587048EE000000007010101010102C
:10484000107C00000000000000FF494949ED000015
:104850000000000000D8664242E7000000000000AF
:10486000003C4242423C00000000000000F846428A
:10487000427C40E000000000003E4242423E02070F
:104880000000000000EE302020F8000000000000D2
:10489000003E403C427C000000000010107C1010E4
:1048A000100C00000000000000C64242423F000021
:1048B0000000000000E7462428100000000000006F
:1048C00000D7929A6A44000000000000006E3C1875
:1048D0003C7600000000000000E74624181810E0B5
:1048E00000000000007E4418327E0000000704042F
:1048F0000408040404040300080808080808080859
:10490000080808080070101010081010101060003F
:10491000304C030000000000000000000000000018
:104920000000000000000000000000000000000087
:104930000000000000000000070007000700020060
:1049400002000200000007000000000000000660F6
:104950000CC0330000000000000000000000000058
:104960000000000000000000104010407FE01040F8
:1049700020807FE0208020800000000000000200F6
:104980001F8032C032000E00038002C032C01F8080
:104990000200000000000000708089808900720021
:1049A00005C00A20122021C0000000000000000005
:1049B0001C002600240019C07880CD00C6007DE0D0
:1049C0000000000000003800080030000000000077
:1049D0000000000000000000000000000000004097
:1049E00000800300060006000600060003000180A8
:1049F000004000000000200018000C000600060027
:104A0000060006000C001800200000000000000056
:104A10000000030062301AC01FC0623006000000B0
:104A200000000000000000000200020002007FF011
:104A30000200020002000000000000000000000070
:104A4000000000000000000000000000000038002E
:104A500008003000000000000000000000007FE0BF
:104A60000000000000000000000000000000000046
:104A700000000000000000000000000000003800FE
:104A80000000000000000020004000800100020043
:104A9000040008001000200040000000000000009A
:104AA0001F8030C0606060606060606030C01F80E8
:104AB000000000000000000002003E0006000600AA
:104AC0000600060006003FC00000000000000000D5
:104AD0001F8061C060C0018002000C0030407FC0B8
:104AE00000000000000000003F00618001800E0017
:104AF000018000C061C03F00000000000000000015
:104B0000018007800980118061801FC0018003C07F
:104B100000000000000000003FC0200020002F80A7
:104B200010C000C061C03F00000000000000000095
:104B30000F8030C060006FC07060606030601F80A8
:104B400000000000000000003FE020400080010065
:104B50000200020006000600000000000000000045
:104B60003FC060E060601F8031C0606070601F8087
:104B700000000000000000001F8070C0606070E056
:104B80003F6000E031C01F00000000000000000096
:104B90000000000007000000000000000000070007
:104BA00000000000000000000000000000000600FF
:104BB0000000000000000600060000000000006089
:104BC000008003000C003000080006000180006037
:104BD0000000000000000000000000007FE0000076
:104BE00000007FE000000000000000000000300036
:104BF0000800060001800060008003000C00300007
:104C000000000000000000001F8060E0606000C045
:104C10000700040000000E0000000000000000007B
:104C20000FC0382063D0649069906FE038000FE0C7
:104C3000000000000000000006000F000B001180C3
:104C400011803FC060C0F1F00000000000000000D3
:104C5000FF8060C060C07F0060C0606060E0FF8077
:104C600000000000000000000FE03820600060003D
:104C70006000600030201FC0000000000000000045
:104C8000FF0060C0606060606060606060C0FF00E6
:104C90000000000000000000FFC0602061007F00F5
:104CA000610060006020FFC0000000000000000004
:104CB000FFC0602061007F00610060006000F000C4
:104CC000000000000000000007C0384060006000E5
:104CD00063F060C030C00F00000000000000000062
:104CE000F0F0606060607FE0606060606060F0F0E5
:104CF00000000000000000003FC0060006000600A3
:104D00000600060006003FC0000000000000000092
:104D10000FF00180018001800180018001806180AD
:104D20003F00000000000000F1E0608067007C00B0
:104D30006200610060C0F0F00000000000000000B0
:104D4000F000600060006000600060006020FFC054
:104D50000000000000000000F0F070E07960596091
:104D60005E604E604C60E4F0000000000000000057
:104D7000E070702058204620432041E04060E02051
:104D800000000000000000001F8030C06060606014
:104D90006060606030C01F80000000000000000004
:104DA000FFC0606060607FC0600060006000F00075
:104DB00000000000000000001F8030C060606060E4
:104DC00060606E6031C01F0000E000000000000065
:104DD000FFC0606060607F806300618060C0F070D1
:104DE00000000000000000001FE0602060001F00C5
:104DF00001C0006040E07F80000000000000000073
:104E00007FE08610060006000600060006000F0080
:104E10000000000000000000F070602060206020B2
:104E20006020602060603FC00000000000000000C3
:104E3000F8F030403040188018800D000F00060058
:104E40000000000000000000F77066206240334060
:104E500037803F8019801100000000000000000032
:104E600079E018800D00060007000980104078E006
:104E70000000000000000000F1F020401080090058
:104E80000600060006001F80000000000000000071
:104E90003FC06080010002000400080010203FC0F5
:104EA00000000000000007E004000400040004000B
:104EB000040004000400040007E0000000002000DB
:104EC00010000800080004000200010000800080BB
:104ED0000040000000003F0001000100010001004F
:104EE00001000100010001003F0000000000070078
:104EF00018C00000000000000000000000000000DA
:104F000000000000000000000000000000000000A1
:104F100000000000000000000000FFF000001C0086
:104F20000000000000000000000000000000000081
:104F300000000000000000000000000000001F80D2
:104F400030C01FC060C03FF0000000000000000043
:104F500070003000300037C03860306030603F8013
:104F600000000000000000000000000000001F0022
:104F70007180600070401F80000000000000000091
:104F800001C000C000C01FC070C060C060C03FE072
:104F900000000000000000000000000000000F8082
:104FA00030603FE030000FC0000000000000000053
:104FB00007E00C000C007FC00C000C000C003F80D0
:104FC00000000000000000000000000000000FF0E2
:104FD00030C01F8030003F8060603FC00000000094
:104FE000700030003000378038C030C030C079E009
:104FF00000000000000000000600000000003E006D
:105000000600060006003FC000000000000000008F
:105010000180000000000F8001800180018001807C
:1050200001803F000000000070003000300033C0FD
:1050300033003E00310079E0000000000000000075
:105040003E000600060006000600060006003FC0FF
:105050000000000000000000000000000000FFE071
:10506000666066606660F770000000000000000087
:10507000000000000000770038C030C030C079E088
:1050800000000000000000000000000000001F8081
:1050900070E0606070E01F80000000000000000011
:1050A00000000000000077C03860306030E03F80D2
:1050B00030007C00000000000000000000001FC065
:1050C00070C060C060C03FC000C003E000000000CE
:1050D000000000000000F9E01E0018001800FF00AA
:1050E00000000000000000000000000000001FE0C1
:1050F00030000F8020603FC0000000000000000072
:10510000000004000C007F800C000C000C400380A9
:10511000000000000000000000000000000071C05E
:1051200030C030C030C01FE00000000000000000B0
:1051300000000000000078F0104008800500020028
:105140000000000000000000000000000000F7B0B8
:10515000632037E03DC01880000000000000000020
:105160000000000000007FE01D80060019807FE045
:10517000000000000000000000000000000079E0D6
:10518000108019000F000600040038000000000025
:105190000000000000003FC02300060018203FE090
:1051A00000000000000001C0010001000100060035
:1051B000010001000100010000C000000200020027
:1051C00002000200020002000200020002000200CF
:1051D0000200020000003800080008000800060075
:1051E0000800080008000800300000003C004710DC
:1051F00001E00000000000000000000000000000CE
:105200000000000000100000001401400100000038
:10521000000800000014014002000000000400002B
:1052200000140140030000000020000000140140B1
:105230000700000000010000001401400800000009
:1052400000800000000C0140040000000800000085
:10525000000C014005000000008000000014014027
:105260000900000000C1814001C0804101C08041AF
:1052700000C1814001C0804100C1814000C1814026
:1052800001C0804101C0804100C1814000C1814016
:1052900001C0804100C1814001C0804101C0804106
:1052A00000C1814001C0804100C1814000C18140F6
:1052B00001C0804100C1814001C0804101C08041E6
:1052C00000C1814000C1814001C0804101C08041D6
:1052D00000C1814001C0804100C1814000C18140C6
:1052E00001C0804101C0804100C1814000C18140B6
:1052F00001C0804100C1814001C0804101C08041A6
:1053000000C1814000C1814001C0804101C0804195
:1053100000C1814001C0804100C1814000C1814085
:1053200001C0804100C1814001C0804101C0804175
:1053300000C1814001C0804100C1814000C1814065
:1053400001C0804101C0804100C1814000C1814055
:1053500001C0804100C1814001C0804101C0804145
:1053600000C1814000C0C101C30302C2C60607C715
:1053700005C5C404CC0C0DCD0FCFCE0E0ACACB0B85
:10538000C90908C8D81819D91BDBDA1A1EDEDF1FB5
:10539000DD1D1CDC14D4D515D71716D6D21213D3A5
:1053A00011D1D010F03031F133F3F23236F6F73755
:1053B000F53534F43CFCFD3DFF3F3EFEFA3A3BFB45
:1053C00039F9F83828E8E929EB2B2AEAEE2E2FEFF5
:1053D0002DEDEC2CE42425E527E7E62622E2E32365
:1053E000E12120E0A06061A163A3A26266A6A76795
:1053F000A56564A46CACAD6DAF6F6EAEAA6A6BAB05
:1054000069A9A86878B8B979BB7B7ABABE7E7FBF34
:105410007DBDBC7CB47475B577B7B67672B2B37324
:10542000B17170B0509091519353529296565797D4
:10543000559594549C5C5D9D5F9F9E5E5A9A9B5BC4
:1054400099595898884849894B8B8A4A4E8E8F4F74
:105450008D4D4C8C448485458747468682424383E4
:105460004181804084540008000000205400000066
:105470006C010008D854000854000020BC2F000024
:10548000880100080000000000000000000000008B
:105490000024F400000000000000000000000000F4
:1054A00000000000100000000100000000000000EB
:1054B00000000000000000000000000000000000EC
:1054C00000000000000000000000000000000000DC
:0854D0000000000000000000D4
:0400000508000131BD
:00000001FF
